:1015EC005343532D34303000020800000244656D23
:1015FC00616E643000010000020800000244656D59
:10160C00616E643100010002020800000244656D45
:10161C00616E643200010004020800000244656D32
:10162C00616E643300010006020800000244656D1F
:10163C00616E643400010008020800000244656D0C
:10164C00616E64350001000A020800000244656DF9
:10165C00616E64360001000C020800000244656DE6
:10166C00616E64370001000E040800000154656DC2
:10167C007030000000010010040800000154656D7A
:10168C007031000000010014040800000154656D65
:10169C007032000000010018040800000154656D50
:1016AC00703300000001001C040800000154656D3B
:1016BC007034000000010020040800000154656D26
:1016CC007035000000010024040800000154656D11
:1016DC007036000000010028040800000154656DFC
:1016EC00703700000001002C045A000001435072B6
:1016FC006F70300000010030045A0000014350723A
:10170C006F70310000010034045A00000143507224
:10171C006F70320000010038045A0000014350720F
:10172C006F7033000001003C045A000001435072FA
:10173C006F70340000010040045A000001435072E5
:10174C006F70350000010044045A000001435072D0
:10175C006F70360000010048045A000001435072BB
:10176C006F7037000001004C045A00000143496EB1
:10177C007430000000010050045A00000143496E0F
:10178C007431000000010054045A00000143496EFA
:10179C007432000000010058045A00000143496EE5
:1017AC00743300000001005C045A00000143496ED0
:1017BC007434000000010060045A00000143496EBB
:1017CC007435000000010064045A00000143496EA6
:1017DC007436000000010068045A00000143496E91
:1017EC00743700000001006C045A00000150496E6F
:1017FC007430000000010070045A00000150496E62
:10180C007431000000010074045A00000150496E4C
:10181C007432000000010078045A00000150496E37
:10182C00743300000001007C045A00000150496E22
:10183C007434000000010080045A00000150496E0D
:10184C007435000000010084045A00000150496EF8
:10185C007436000000010088045A00000150496EE3
:10186C00743700000001008C045A000001506F779F
:10187C006572300000010090045A000001506F772F
:10188C006572310000010094045A000001506F771A
:10189C006572320000010098045A000001506F7705
:1018AC00657233000001009C045A000001506F77F0
:1018BC0065723400000100A0045A000001506F77DB
:1018CC0065723500000100A4045A000001506F77C6
:1018DC0065723600000100A8045A000001506F77B1
:1018EC0065723700000100AC02080000024F6673FD
:1018FC0030000000000100B002080000024F6673C7
:10190C0031000000000100B202080000024F6673B3
:10191C0032000000000100B402080000024F6673A0
:10192C0033000000000100B602080000024F66738D
:10193C0034000000000100B802080000024F66737A
:10194C0035000000000100BA02080000024F667367
:10195C0036000000000100BC02080000024F667354
:10196C0037000000000100BE020300000050657249
:10197C00696F6400000100C000000000000000005E
:08198C00000000000000000053
:0E2E7F00011D010363FF15F401500001550011
:1027020075A490E4F5BA75BCE075E88075D10375DF
:10271200D48075D78075A5FFEF6079E4FBEB25E0E7
:1027220025E02490F582E43400F583120EDF0000E8
:1027320000000BBB08E7E4FBEB25E02400F582E494
:102742003400F583E4F0A3F0EB25E025E02430F536
:1027520082E43400F583120EDF3F800000EB25E0B7
:1027620025E02450F582E43400F583120EDF3DCCDF
:10277200CCCDEB25E025E02470F582E43400F5832E
:10278200120EDF000000009000C0E4F0A3743CF0E1
:042792000BBB08A4D1
:012796002220
:092EC9001510A810EFF605102207
:050003008F347F002294
:102D29008B348A358936120C3BAB37AA38A939124C
:102D39000C81AB34AA35A936900001120C54AB377B
:0D2D4900AA38A939900001120C937F0222D4
:10232B00E5557017E550045407F550540FF5BB7580
:10233B00BCE0E4F554F553F552F551E4F53AC2AF70
:10234B00C2EDD2EC30EDFDD2AFAFBFEFFEADBEEDC7
:10235B00FFE4FCFDE5542FF554E5533EF553ED3505
:10236B0052F552EC3551F551122A20053AE53AC394
:10237B00941040CA0555E5556003022421AF54AEB5
:10238B0053AD52AC51FB7A01F9F8120DF18F548E0B
:10239B00538D528C51E4120B7CE4FBFA7980784715
:1023AB00120A72E4FBFA79FA78431209698F3E8EAE
:1023BB003D8D3C8C3BAB3EAA3DA93CA83BE8C0E025
:1023CB00E9C0E0EAC0E0EBC0E0E55025E024B0F561
:1023DB0082E43400F583E0FCA3E0FDEC120B81E416
:1023EB00FBFA79C87842120A72D0E0FBD0E0FAD03F
:1023FB00E0F9D0E0F81208788F3E8E3D8D3C8C3B97
:10240B00C2AFE55025E025E02410F582E43400F559
:06241B0083120EBAD2AFDD
:012421002298
:101ED600122EB5AB5DAA5CA95BA85AC3120E91700F
:101EE6000302211C122EB58F5D8E5C8D5B8C5AE42D
:101EF600F53AE53A25E025E02490F582E43400F54C
:101F060083E0FCA3E0FDA3E0FEA3E0FFE4FBFA7997
:101F1600C87842120B0F6002500302207A122EB5C7
:101F2600C3EF9559F542EE9558F541ED9557F540B5
:101F3600EC9556F53FE53A25E025E02490F582E458
:101F46003400F583E0FCA3E0FDA3E0FEA3E0FF126E
:101F56000BBAAB42AA41A940A83FC3120E91500347
:101F660002207AE53A25E025E02490F582E4340063
:101F7600F583E0FCA3E0FDA3E0FEA3E0FF120BBAAD
:101F8600E4120B7CC8ECC8C9EDC9CAEECACBEFCBCC
:101F9600E53A25E025E02490F582E43400F583E077
:101FA600FCA3E0FDA3E0FEA3E0FF1208748F3E8EC3
:101FB6003D8D3C8C3BE4FFFEFDFCAB3EAA3DA93CBF
:101FC600A83B120B0F6038E53A25E025E02490F592
:101FD60082E43400F583E0FCA3E0FDA3E0FEA3E089
:101FE600FF120BBAEF2401FFE43EFEE43DFDE43CA4
:101FF600FCAB42AA41A940A83FC3120E914010AFC4
:102006003A7401C8EFC8088002C333D8FC805AE589
:1020160062D3940040587466253AF8E6FCE4120B45
:1020260086ECC0E0EDC0E0EEC0E0EFC0E0AC62E4FC
:10203600120B86C8ECC8C9EDC9CAEECACBEFCBD025
:10204600E0FFD0E0FED0E0FDD0E0FC120A72AB3E2D
:10205600AA3DA93CA83B120B0F5013AF3A7401C816
:10206600EFC8088002C333D8FCF452908006746629
:10207600253AF806053AE53AC394085003021EF8D5
:10208600122EB5C3EF9559FFEE9558FEED9557FD07
:10209600EC9556FCE47B64FAF9F8D3120E9150766F
:1020A600122EB58F598E588D578C568F5D8E5C8D3E
:1020B6005B8C5AE4F53AE53A25E025E02490F58272
:1020C600E43400F583E0FCA3E0FDA3E0FEA3E0FF1B
:1020D600E4FBFAF9F8120B0F5010AF3A7401C8EF8F
:1020E600C8088002C333D8FC4290053AE53AB408E2
:1020F600C5E5622401FFE433FE7C007D0A120CC7AD
:102106008D62E5627010F53A7466253AF8E4F605D4
:062116003AE53AB408F2BC
:01211C0022A0
:101C49009000C0E07002A3E07003021ED5122EB509
:101C5900ECC0E0EDC0E0EEC0E0EFC0E09000C0E015
:101C6900FEA3E0FF7C007D64120CB5EF2561FBEE5D
:101C79003560FAE4355FF9EC355EF8D0E0FFD0E085
:101C8900FED0E0FDD0E0FCC3120E914003021ED548
:101C9900122EB58F618E608D5F8C5EE4F53AE53A60
:101CA90025E025E02470F582E43400F583C083C083
:101CB90082E0F8A3E0F9A3E0FAA3E0FBE8C0E0E9D9
:101CC900C0E0EAC0E0EBC0E0E53A25E02400F58297
:101CD900E43400F583E0FCA3E0FDEC120B81E53A66
:101CE90025E025E02410F582E43400F583E0F8A32B
:101CF900E0F9A3E0FAA3E0FB120874E53A25E02530
:101D0900E02450F582E43400F583E0F8A3E0F9A378
:101D1900E0FAA3E0FB120969D0E0FBD0E0FAD0E0D9
:101D2900F9D0E0F8120878D082D083120EBAE53AD9
:101D390025E025E02470F582E43400F583E0FCA376
:101D4900E0FDA3E0FEA3E0FFE4FBFAF9F8120B0FB4
:101D590060184016E53A25E025E02470F582E43460
:101D690000F583120EDF00000000E53A25E025E0CA
:101D79002470F582E43400F583E0FCA3E0FDA3E0E0
:101D8900FEA3E0FFE4FBFA79C87842120B0F501664
:101D9900E53A25E025E02470F582E43400F5831264
:101DA9000EDF42C80000E53A25E025E02470F582FF
:101DB900E43400F583E0FCA3E0FDA3E0FEA3E0F535
:101DC9003E8E3D8D3C8C3BFBAA3DA93CA83BE8C01F
:101DD900E0E9C0E0EAC0E0EBC0E0E53A25E0240034
:101DE900F582E43400F583E0FCA3E0FDEC120B81FD
:101DF900E53A25E025E02410F582E43400F583E096
:101E0900F8A3E0F9A3E0FAA3E0FB120874E53A2588
:101E1900E025E02430F582E43400F583E0F8A3E01E
:101E2900F9A3E0FAA3E0FB120969D0E0FBD0E0FADC
:101E3900D0E0F9D0E0F81208788F3E8E3D8D3C8CC9
:101E49003BE4FFFEFDFCAB3EAA3DA93CA83B120BBF
:101E59000F5009E4F53EF53DF53CF53BE4FFFE7D09
:101E6900C87C42AB3EAA3DA93CA83B120B0F600DB2
:101E7900400BE4F53EF53D753CC8753B42E4FFFE79
:101E89007D207C41AB3EAA3DA93CA83B120969E4EF
:101E9900FBFAF9783F120878120BBACDEFCDCCEEE8
:101EA900CCEC120B81E4FBFA79207841120A72E535
:101EB9003A25E025E02490F582E43400F583120EFA
:0C1EC900BA053AE53A64086003021CA761
:011ED50022EA
:092ED20012232B121C49021ED62A
:0D2E9100245265763A203439313620240071
:10199400E47880F612000EC2B575E104E4F5E27550
:1019A400E34075A401F5A5F5A675A72075B1677583
:1019B400B208122E63E4FF122E4443EF04E4F53C14
:1019C400F53D7D01AF3D122DD7053DE53D70020586
:1019D4003CC39401E53C940040E8E4F520C20AC20B
:1019E40008C20EC20DC20C7880F608F67885F61887
:1019F400F6788AF6F53CF53D74A2253DF8E4F60543
:101A04003DE53D7002053C6414453C70EBE4F53C57
:101A1400F53D74B6253DF8E4F6053DE53D70020557
:101A24003C6408453C70EBE5EF20E10CE5EF54081D
:101A3400D394004003D38001C392037D08E4FF12D2
:101A44002DFEE47889F67882F6AB63AA64A96578FA
:101A540082E6FF75F010A4F58285F083120C54FE23
:101A6400788926F6EE600578820680DDEFD394004F
:101A74004030AB63AA64A96590000D120F10120CDC
:101A84003BFF7455120C81120C3B64556002D20C5E
:101A940074AA120C81120C3B64AA6002D20CEF12DD
:101AA4000C81E5EF5402D3940040047F018002E4EA
:101AB400FF1224228F3BE53B20E036C20974FF78F5
:101AC4008CF608F608F608F67E007F107D007B0091
:101AD4007A007992120F667541FF7542157543ECD1
:101AE4007544007545107B007A007992122BFD80B5
:101AF40002D209902E98E493FF3395E0FEEF24D0B0
:101B0400FFEE34FFFE7C007D64120CB5AA06AB0721
:101B1400902E97E493FF3395E0FEEF24D0FFEE344C
:101B2400FFFE7C037DE8120CB5EF2BFBEE3AFA9036
:101B34002E99E493FF3395E0FEEF24D0FFEE34FFBB
:101B4400FE7C007D0A120CB5EF2BFFEE3AFEA3E4F7
:101B540093FD3395E0FCED24D0FDEC34FFCD2F78DC
:101B640091F6ED3E18F6E53B30E103021C20E4F566
:101B74003CF53DE53DC4F8540FC868FFE53CC4544A
:101B8400F048FEAB63AA64A9658F82F583120C54F6
:101B94007003021C17E92FF9EA3EFA900004120CB4
:101BA4005420E264E4F53AE53AC3781D965059E5C9
:101BB4003DC4F8540FC868FFE53CC454F048AB6317
:101BC400AA64A9658F82F583120C54FF7E00C006B7
:101BD400C0077D00E53DC4F8540FC868FFE53CC468
:101BE40054F048FEE92FF9EA3EFA90000D120F1066
:101BF4007889E6853AF0A429F9EA35F0FAD007D0D5
:101C040006120F66053A809F053DE53D7002053CCE
:101C1400021B777F01122702C20B8007E4FF122701
:101C240002D20BE4F53CF53D7A007B967D03AF3D93
:101C3400122935053DE53D7002053CC39401E53CA0
:041C4400940040E4E4
:011C48002279
:052EDB00788AE6FF22E9
:030023000222278F
:10222700C0E0C0F0C083C082C0D075D000C000C07D
:1022370001C002C003C004C005C006C00730993AF8
:10224700C2997885067985E77881667016F678856C
:01225700F690
:0E22580075220A0075230300D523FCD522F55C
:04226600C2B5801766
:0E226A007522140075230300D523FCD522F540
:102278007885E624B6F8E6F599209803022310201D
:102288009A07200A04C298807BC29A7884E60624BA
:10229800A2F8A699C2987884E6FFB4011378A2E65A
:1022A800FE70057884F68060EE54072402788BF679
:1022B800EFB4020E788BE6B4090878A3E624037914
:1022C8008BF77884E6FFB414047600803BEFC3787C
:1022D8008B9640347884E624FFFDE434FFFC7B00D1
:1022E8007A0079A21227977884E624A1F8E66F602D
:0322F80002801150
:0E22FB007522140075230300D523FCD522F5AF
:1023090012002678847600D007D006D005D004D0F4
:1023190003D002D001D000D0D0D082D083D0F0D069
:02232900E032A0
:1029AE0078A3E675F010A4AB632565F9E56435F000
:1029BE00FA90000D120F10788AE6FF18E68FF0A439
:1029CE002526F582E435F0F583120C54FF7B007A50
:0329DE0000792459
:1029E1008F348B358A368937EA494B6016120C3B96
:1029F100FFE534FD7C00122E9EAB35AA36A937EFD8
:032A0100120C8133
:0E2A04007538140075390300D539FCD538F546
:0E2A12008534997F01122D563099FDC299220C
:102DAD0078B676787884E624A1F8E678B7F67F02CF
:062DBD007881EFF6D2B5AB
:0E2DC3007534140075350300D535FCD534F594
:062DD10078B6E6F5992238
:102CA000C9EFC9E964017028EDC39B4034781DE683
:102CB000FFEB2FFFE433FEEDC39FEE6480F87480DA
:102CC00098501ED20AC3ED9B788AF6788676012248
:102CD000B90214ED6B700AD20A788AF67886760209
:082CE00022C20AE47886F62204
:102AF300C9EFC9BAFF15BBFF12ED6B7002EC6A7028
:102B030049D20A788AF67886E9F622E964017025C3
:102B1300C3ED9BEC9A401C781DE62BFFE43AFEC301
:102B2300ED9FEC9E500DD20AC3ED9B788AF6788612
:102B33007601228015B90218ED6B7002EC6A700AF7
:102B4300D20A788AF67886760222C20AE47886F672
:012B5300225F
:1000260078A2E6FF54F8F525EF120F40006F09009D
:100036007B0A008D1000961100A61200BC1900D193
:100046001A00F32000F928017B29027F3302B73713
:1000560002DD3902F64102FF49030850034C6102F2
:1000660045700344980000037778A3E6FD788DE693
:10007600FB7F01802578A3E6FC08E6FD788CE6FA8E
:1000860008E6FB7F018029D20A7886760302037789
:1000960078A3E6FD788FE6FB7F02122CA002037799
:1000A60078A3E6FC08E6FD788EE6FA08E6FB7F0212
:1000B600122AF302037778A3E6FD788DE6FB7F012B
:1000C600122CA0200A03020377801978A3E6FC0805
:1000D600E6FD788CE6FA08E6FB7F01122AF3200A91
:1000E6000302037778B676787F0102037475EF1002
:1000F600020377C2ACE4F524D2B5FB7A0079247FFB
:100106007F1229E17B007A0079247F181229E17B8E
:10011600007A0079247F051229E17882E61229DA2D
:10012600788CE61229DA788DE61229DA788EE612CC
:1001360029DA788FE61229DA7890E61229DA7891A8
:10014600E61229DAE4F52674922526F8E61229DA6B
:100156000526E526C3941040EE7B007A007900AFB1
:04016600241229E155
:0E016A0075320A0075330300D533FCD532F52B
:1001780002023278A3E6FFC378829640030202396E
:10018800EF75F010A42565F9E56435F085632FF562
:10019800308931C2ACE4F524D2B5FB7A0079247FEA
:1001A8007F1229E17B007A0079247F0D1229E1ABC7
:1001B8002FAA30A931120C3B1229DAAB2FAA30A989
:1001C800319000011229D7AB2FAA30A93190000233
:1001D8001229D7AB2FAA30A9319000031229D7AB27
:1001E8002FAA30A9319000041229D7E4F526AB2FA5
:1001F800E5312405F9E43530FA7E00E92526F9EEE3
:100208003AFA120C3B1229DA0526E526C39408406F
:0C021800DD7B007A007900AF241229E1A0
:0E02240075320A0075330300D533FCD532F570
:10023200C2B5D2AC02037778B67678E408F67F02CC
:10024200020374122EBF7811120EAE78B6767C7845
:1002520011E678B7F67812E678B8F67813E678B948
:10026200F67814E678BAF67C007D057B007A007990
:10027200B612279778BBEFF67F0602037478A3E6DF
:10028200FFB4010F08E6FD08E6788CCDF608EDF61E
:10029200020344EFB4020978A4E6788CF602034420
:1002A20078A3E6B4030C08E6FF08E6788ECFF608DA
:1002B200EFF6020344E4F526E526C378A39650152B
:1002C20074A42526F8E6FF74922526F8EFF6052693
:1002D200E526B410E3E478A1F680677A007B327DEC
:1002E20001788AE6FF12293578A3E6FDE4FF122D94
:1002F200FE02037778A3E624FF9202807878A3E6D1
:1003020024FF9201806F788AE66005752802800BCF
:10031200200D05752803800375280178B6767908C3
:10032200A6287C007D027B007A0079B61227977896
:10033200B8EFF67F03122DBDE52864017037D20EA7
:100342008002D208788076F1802B7A007B327D01A0
:100352007F0012293578B6767978A3E678B7F67CED
:10036200007D027B007A0079B612279778B8EFF603
:100372007F03122DBDE52564A0600302057578A2F6
:10038200E664A1600302046F79A3E7C37882964012
:1003920003020466AB63AA64A96578A3E6FF75F05D
:1003A20010A4F58285F083120C54F528EF75F01035
:1003B200A429F9EA35F0FA900004120C5430E23024
:1003C20078A3E6FF1200038F2878B6767F08A62866
:1003D200E5282402FDE433FC7B007A0079B612277B
:1003E2009774B82528F8EFF6E5282403FF02057272
:1003F20078A3E6FF120003C2ACE4F524D2B5E528E7
:10040200D39406402B7B007A0079247F7F1229E166
:100412007B007A007924AF281229E1E4F526E5264B
:10042200C3952850071229AE052680F205288018A8
:10043200E52824781229DAE4F526E526C395285022
:10044200071229AE052680F27B007A007900AF24DC
:030452001229E18B
:0E04550075320A0075330300D533FCD532F53D
:1004630002056678B676787F0102057278A2E664A3
:10047300A260030205757882E6FF78A3E6FEC39FB8
:10048300400302056C08E6FDC39F400302056CEEC2
:100493009D400302056C18E6F526E4F52DF52EE5DF
:1004A30026D378A4965026AF26120003AB63AA6422
:1004B300A96575F010E526A4F58285F083120C5426
:1004C300252EF52EE4352DF52D052680D2C2ACE47C
:1004D300F524D2B5FB7A0079247F7F1229E1C3E5A5
:1004E3002E9480E52D940050028007E52D44801260
:1004F30029DAAF2E1229DB78A3E6F526E526D37891
:10050300A4965046E4F527AB63AA64A96575F01079
:10051300E526A4F58285F083120C54FFE527C39FDB
:100523005024E52675F010A429F9EA35F0FA900075
:100533000D120F10788AE6FF18E68FF0A425271214
:1005430029D0052780C1052680B27B007A00790077
:05055300AF241229E1B4
:0E05580075320A0075330300D533FCD532F539
:10056600C2B5D2AC800978B676787F01122DBDE58A
:100576002564587047FA7B327D01788AE6FF122996
:10058600357537007538007539B77B007A0079A361
:10059600122D298F28E528247878B6F6E528240137
:1005A600FDE433FC7B007A0079B612279774B725F1
:1005B60028F8EFF6E5282402FF122DBDE525648014
:1005C6006009E5256488600302074C7886E6B40175
:1005D6000F7A007B327D01788AE6FF122935801A70
:1005E600E4F526E526C3781D96500F7A007B327D0A
:1005F60001AF26122935052680E978A2E65407F5CB
:1006060028B4070A75270108E6F528088005E4F5E9
:100616002778A3E6F5291528E529C37882964003AD
:1006260002073AAB63AA64A96575F010E529A4F53B
:100636008285F083120C54FFE528D39F40028F2851
:100646007886E6B40109788AE6F52CF52B8009E46C
:10065600F52B781DE614F52C788AA62B788AE6D336
:10066600952C400302072EE4F526E526C39528407F
:1006760003020723E52975F010A4AB632565F9E5A8
:100686006435F0FA900004120C5430E20302071E9F
:10069600900001120C5464387031E528D39404405C
:1006A6000BE527252624A4F8E6FD804E7884E6C3CC
:1006B6009526FF74A02FF8E6FDE52975F010A4AB8A
:1006C600632565F9E56435F0FA802FAB63AA64A962
:1006D6006575F010E529A4F58285F083120C54FFA8
:1006E600C37884E69F2526252724A1F8E6FDE5297B
:1006F60075F010A429F9EA35F0FA90000D120F10E2
:10070600788AE6FF18E68FF0A4FFE5262FF582E447
:1007160035F0F583ED120C930526020670AF29120B
:100726002EC9788A06020662788AA62BE525648891
:100736007014800FE529B4FF0D78A4E6F520E525B1
:10074600B48803122DADE52564A86003020870780D
:1007560086E6B4010F7A007B327D01788AE6FF12C5
:100766002935801AE4F526E526C3781D96500F7ABA
:10077600007B327D01AF26122935052680E978A354
:10078600E630E711547FFE08E6FDEEF52DEDF52E79
:10079600752703800B78A3E6752D00F52E752702C5
:1007A60074A22527F8E6FF74A32527F8E6F52A8F15
:1007B60029E529D3952A400302086DE529C37882E5
:1007C600964003020868AB63AA64A96575F010E554
:1007D60029A4F58285F083120C54F5287886E6B4B0
:1007E6000109788AE6F52CF52B8009E4F52B781DAE
:1007F600E614F52C788AA62B788AE6D3952C5058E1
:10080600E4F526E526C395285044E52975F010A49D
:10081600AB632565F9E56435F0FA900004120C54D3
:1008260020E227E527252624A4F8E6FD90000D12F0
:100836000F10788AE6FF18E68FF0A4FFE5262FF55D
:1008460082E435F0F583ED120C93052680B5AF29C9
:10085600122EC9788A0680A0788AA62BE528252735
:0A086600F52705290207B7122DAD92
:010870002265
:100FCF007880E664F160030215EBE4F544F54578AB
:040FDF0081E6602027
:0E0FE300754A0A00754B0300D54BFCD54AF544
:100FF1000545E5457002054464107004E544642725
:1010010070DBC2AF75FFDE75FFADE4F540F53F2043
:10101100982FE4F544F545209823C3E5459488E5E8
:05102100449413501877
:0E102600754A0A00754B0300D54BFCD54AF500
:101034000545E54570DE054480DAB2B480CE859975
:101044003FC298E53F641A6003021119F544F5455F
:0E105400209823C3E5459488E5449413501872
:0E106200754A0A00754B0300D54BFCD54AF5C4
:101070000545E54570DE054480DA30989385994052
:10108000C298E4F544F545209823C3E5459488E5E6
:05109000449413501808
:0E109500754A0A00754B0300D54BFCD54AF591
:1010A3000545E54570DE054480DA209803021010FB
:1010B300859940C298E4F544F545209823C3E54556
:0810C3009488E54494135018D1
:0E10CB00754A0A00754B0300D54BFCD54AF55B
:1010D9000545E54570DE054480DA209803021010C5
:0910E900859940C298D2B5C29964
:0E10F200754A1400754B0300D54BFCD54AF52A
:061100007599783099FD9D
:0E110600754A0A00754B0300D54BFCD54AF51F
:10111400C2B50215DDE53F645060030211AEF5442B
:10112400F545209823C3E5459488E5449413501865
:0E113400754A0A00754B0300D54BFCD54AF5F1
:101142000545E54570DE054480DA2098030210105B
:09115200859940C298D2B5C299FA
:0E115B00754A1400754B0300D54BFCD54AF5C0
:081169007599793099FDC299D6
:0E117100754A1400754B0300D54BFCD54AF5AA
:08117F007599013099FDC29938
:0E118700754A1400754B0300D54BFCD54AF594
:06119500E4F5993099FD1C
:0E119B00754A0A00754B0300D54BFCD54AF58A
:0F11A900C2B50215DDE53F64017041D2B5C299B0
:0E11B800754A1400754B0300D54BFCD54AF563
:0811C6007599783099FDC2997A
:0E11CE00754A1400754B0300D54BFCD54AF54D
:0611DC00E4F5993099FDD5
:0E11E200754A0A00754B0300D54BFCD54AF543
:1011F000C2B50215DDE53F640260030212B7F54493
:10120000F545209823C3E5459488E5449413501888
:0E121000754A0A00754B0300D54BFCD54AF514
:10121E000545E54570DE054480DA2098030210107E
:10122E00859940C298E4F541E54013B392B4E54088
:10123E0025E0FEC3E494CFEE940F5029E5407F00E5
:10124E0025E0FEC39460501DE5B654F04408F5B693
:10125E00758F038E468F478547828E83E4F053B693
:0C126E00F0F58F80037541FFD2B5C299E6
:0E127A00754A1400754B0300D54BFCD54AF5A0
:081288007599783099FDC299B7
:0E129000754A1400754B0300D54BFCD54AF58A
:06129E008541993099FD25
:0E12A400754A0A00754B0300D54BFCD54AF580
:1012B200C2B50215DDE53F64036003021404F54480
:1012C200F545209823C3E5459488E54494135018C6
:0E12D200754A0A00754B0300D54BFCD54AF552
:1012E0000545E54570DE054480DA209803021010BC
:1012F000859940C298E4F544F545209823C3E54517
:081300009488E5449413501891
:0E130800754A0A00754B0300D54BFCD54AF51B
:101316000545E54570DE054480DA20980302101085
:10132600859942C298E5401392B4E54025E0FEC394
:10133600E494CFEE940F4003021010E5407D0025A3
:10134600E0FCC394604003021010E5B654F0440874
:10135600F5B6758F01E54275F020A42DFFE5F03C4A
:10136600F5468F47E4F543E543C394205049E4F539
:1013760044F545209823C3E5459488E544941350E5
:01138600184E
:0E138700754A0A00754B0300D54BFCD54AF59C
:101395000545E54570DE054480DA20980302101006
:1013A5000547E547AE467002054614F5828E83E58E
:1013B50099F0C298054380B053B6F0E4F58FD2B5E5
:0213C500C299CB
:0E13C700754A1400754B0300D54BFCD54AF552
:0813D5007599783099FDC29969
:0E13DD00754A1400754B0300D54BFCD54AF53C
:0613EB00E4F5993099FDC4
:0E13F100754A0A00754B0300D54BFCD54AF532
:1013FF00C2B50215DDE53F640460030214B8F5447D
:10140F00F545209823C3E5459488E5449413501877
:0E141F00754A0A00754B0300D54BFCD54AF503
:10142D000545E54570DE054480DA2098030210106D
:10143D00859940C298E54025E0F548754900E4F5E9
:10144D0041F544F5450549E549AE48700205481496
:10145D00F5828E83E4932541F5410545E5457002FE
:0E146D0005447004E544640270DBD2B5C299F8
:0E147B00754A1400754B0300D54BFCD54AF59D
:081489007599783099FDC299B4
:0E149100754A1400754B0300D54BFCD54AF587
:06149F008541993099FD22
:0E14A500754A0A00754B0300D54BFCD54AF57D
:1014B300C2B50215DDE53F640560030215D5F544A9
:1014C300F545209823C3E5459488E54494135018C3
:0E14D300754A0A00754B0300D54BFCD54AF54F
:1014E1000545E54570DE054480DA209803021010B9
:1014F100859940C298E4F544F545209823C3E54514
:081501009488E544941350188E
:0E150900754A0A00754B0300D54BFCD54AF518
:101517000545E54570DE054480DA20980302101082
:09152700859942C298D2B5C2991F
:0E153000754A1400754B0300D54BFCD54AF5E7
:08153E0075997F3099FDC299F7
:0E154600754A1400754B0300D54BFCD54AF5D1
:101554007599203099FDE54025E0FCE54275F020C1
:10156400A42400FFE5F03CF5488F49E4F541F54338
:02157400C2991A
:0E157600754A1400754B0300D54BFCD54AF5A1
:10158400854982854883E493F5993099FD0549E5B9
:1015940049AE487002054814F5828E83E4932541D0
:0B15A400F5410543E543B420C7C299A0
:0E15AF00754A1400754B0300D54BFCD54AF568
:0615BD008541993099FD03
:0E15C300754A0A00754B0300D54BFCD54AF55E
:1015D100C2B58008E53FB4060375EF10E53F640727
:0A15E10060030210107880F6D2AF0C
:0115EB0022DD
:102A20007F00122D5620090B7A007B327D017F003A
:102A3000122935300C0B7A007B1E7D017F00122994
:102A400035300817300D147A007B327D01788AE624
:102A5000FF122935C2081225C1D209200B0C300DF6
:102A600009788076F11225C1D20B300E08300D05A1
:102A7000C20E120FCF200D12122EB5E47B2C7A015C
:0B2A8000F9F8C3120E915002D20D2293
:0B2EAA00121994122A20122ED280F878
:10211D00005EBCE2613FDD83C29C7E20A3FD1F41BA
:10212D009DC3217FFCA2401E5F01E3BD3E6082DCAA
:10213D00237D9FC1421CFEA0E1BF5D0380DE3C629A
:10214D00BEE0025CDF81633D7C22C09E1D43A1FF8A
:10215D004618FAA427799BC584DA3866E5BB59077A
:10216D00DB856739BAE406581947A5FB7826C49A6A
:10217D00653BD987045AB8E6A7F91B45C6987A245A
:10218D00F8A6441A99C7257B3A6486D85B05E7B94A
:10219D008CD2306EEDB3510F4E10F2AC2F7193CD3A
:1021AD00114FADF3702ECC92D38D6F31B2EC0E502A
:1021BD00AFF1134DCE90722C6D33D18F0C52B0EE1A
:1021CD00326C8ED0530DEFB1F0AE4C1291CF2D730A
:1021DD00CA947628ABF517490856B4EA6937D58BFA
:1021ED005709EBB536688AD495CB2977F4AA4816EA
:1021FD00E9B7550B88D6346A2B7597C94A14F6A8DA
:10220D00742AC896154BA9F7B6E80A54D7896B35C9
:0A221D00000060B0CBD8E5F3F70035
:032E8D0001730AC4
:1027970015101510A810ECF608EDF6151015101504
:1027A70010A810C6EBC608C6EAC608C6E9C6E510F3
:0427B70024FCF510F9
:1027BB00F80808E4F6A810F608F6E5102407F9A8BF
:1027CB0010E6FE08E6FFC3099719E76480F8EE648C
:1027DB0080985037E5102404F8CBE6CB08E6FA08CE
:1027EB00E6F98F828E83120C54A810080866FFE559
:1027FB00102403F8EFF6E690211D93A8100808F6B5
:10280B00A8100806E61870B20680AFA8100808E6F4
:01281B00FFBD
:07281C00E5102409F510226C
:0B2E9E00ED6F7815F6E690211D93FF04
:012EA9002206
:102DFE00EF701E7598D0E589540F4420F58953C89D
:102E0E00E1438E10ED90221C93F58DD28ED2ACC282
:032E1E00BCD2AF74
:012E2100228E
:102C4F007876120EC600000000787A120EC60000C9
:102C5F000000786E7664E47816F67816E6FFC39473
:102C6F0001502DEF25E025E0246FF8E4F6EF25E085
:102C7F0025E02470F8E4F6EF25E025E02471F8E470
:102C8F00F6EF25E025E02472F8E4F678160680CA00
:012C9F002212
:102E6300D2AFD2A9C2BBE589540F4401F589758E4F
:0C2E730002758CECE4F58AD28C022C4F26
:0226640015104F
:10266600A810E4F6A810E6FFC3940140030226FF73
:10267600EF25E025E02472F8E6FFD394004066A833
:1026860010E625E025E02470F8E67059EF30E015F5
:10269600A810E6FF25E025E02472F8E6D394014071
:1026A600047D0180067D00A810E6FF122CE8A81024
:1026B600E6FF25E025E02472F8E6B401057D001268
:1026C6002CE8A810E6FF25E025E02472F816E6605F
:1026D60014EF25E025E02471F8E6FEEF25E025E07D
:1026E6002470F8EEF6A810E625E025E02470F8E65A
:0926F600600116A8100602266A14
:0326FF00051022A1
:03000B000228AF19
:1028AF00C0E0C0F0C083C082C0D0E8C0E0E9C0E0A3
:1028BF00EAC0E0EBC0E0ECC0E0EDC0E0EEC0E0EF5E
:1028CF00C0E0758CEC7876120EA2EF2401FFE43E87
:1028DF00FEE43DFDE43CFC7876120EAE786E16E613
:1028EF00701B787A120EA2EF2401FFE43EFEE43D46
:1028FF00FDE43CFC787A120EAE786E766412266494
:10290F00122E22D0E0FFD0E0FED0E0FDD0E0FCD0D0
:10291F00E0FBD0E0FAD0E0F9D0E0F8D0D0D082D010
:06292F0083D0F0D0E0327D
:102DD7001510A810EDF61510A810EFF6A810E6FFCD
:102DE700C39401500D08E6FEEF25E025E0246FF8B7
:072DF700EEF60510051022A5
:1029350015101510A810EAF608EBF61510A810EDFD
:10294500F61510A810EFF6A810E6FFC39401505233
:10295500EF25E025E02472F8E67047A810E6FB2590
:10296500E025E02470F8E67039A81008E625E004B3
:10297500FFA810E6FA25E025E02472F8EFF6A81086
:102985000808E6FE08E6FF7C007D0A120D1CEA2514
:10299500E025E02471F8EFF6EB25E025E02470F85A
:0929A500E4F6E5102404F510220B
:102CE8001510A810EDF61510A810EFF6A810E6FFBD
:102CF800C39401501CEF25E025E0246FF8E660112D
:102D0800A81008E670047F0180027F00A81008EF71
:102D1800F6A810E6700608E624FF92B40510051020
:012D28002288
:092EB500C2AF7876120EA2D2AF72
:012EBE0022F1
:092EBF00C2AF787A120EA2D2AF64
:012EC80022E7
:102D56001510A810EFF6A810E670057874F608F6B8
:102D6600300F167873E675F064A4FFC37875E69F96
:0C2D760018E695F0500375FFA50510222B
:102E4400D20FE47874F608F6EF78736003F6800224
:0F2E5400760A75FF0775FFA543B28075EF092257
:10000E00C20FE47874F608F6787376FF75FFDE7526
:03001E00FFAD2211
:102E2200787506E618700106300F167873E675F0AD
:102E320064A4FFC37875E69F18E695F0500375FF0A
:022E4200A522C7
:042D82008E088F091F
:102D8600E4F50AF50BC3E50B9509E50A9508501617
:102D96007FE87E03122B547F01122D56050BE50B9F
:062DA60070E3050A80DF66
:012DAC002204
:042B54008E0C8F0D47
:102B5800D3E50D94FAE50C9400500FEFD3940040A0
:102B680041007E0300DEFD1F80F1850C0E850D0FF0
:102B7800D3E50F94FAE50E940040157FFA7E001213
:102B88002B547406250FF50F74FF350EF50E80E0F3
:102B9800D3E50D9400E50C94004007AF0FAE0E127C
:022BA8002B54AC
:012BAA002208
:102A8B00754A00754B00754C447B007A0079427D8A
:012A9B000238
:082A9C008B468A4789488D49E9
:102AA4007F01122D56AB4AAA4BA94C120D52240099
:102AB400FFE5F03460FE85464D85474E85484FE47A
:102AC400FDEDC39549501BEF2DF582E43EF583E4FB
:102AD40093AB4DAA4EA94F8D82758300120C930DB2
:0F2AE40080DFAB4AAA4BA94CE48549F0020D7D77
:10250A00754112754234754900754A00754B437B13
:07251A00007A0079417D0207
:082521008B458A4689478D486D
:102529007880E664F160030225C012000EC2AFE5AF
:10253900B654F04408F5B6758F01AB49AA4AA94BC0
:10254900120D522400FFE5F034607816F608EFF614
:10255900AA46A947781AA64508C6EAC608C6E9C61A
:10256900E47818F67818E6C395485032781ACBE61D
:10257900CB080806E618CAE6CA70010614F9120C57
:102589003B7819F6E6FF78160806E618CCE6CC7013
:10259900010614F5828C83EFF078180680C6E4F5FD
:1025A9008F53B6F0AB49AA4AA94B8548F0120D7D65
:0725B900D2AFE4FF122E4433
:0125C00022F8
:102BAB007880E664F1704AC2AF12000EE5B654F0BD
:102BBB004408F5B6758F0378177660087600E478CD
:102BCB0016F67817E6FE08E6F5828E83E4F07F01B1
:102BDB00122D567818E426F618740236F61806E607
:102BEB00C3940840DDE4F58F53B6F0D2AFFF122E3D
:012BFB004495
:012BFC0022B6
:1025C100122BABE4F543F544F549754A00754B43CD
:1025D100FB7A00798C7D1612252112250AE4F5403B
:1025E100E540C3781D965073E4F53FAB63AA64A937
:1025F1006575F010E53FA4F58285F083120C5460F7
:1026010056E53F75F010A429F9EA35F0FA90000D6E
:10261100120F107889E68540F0A429F9EA35F0FA1D
:10262100EBC0E0EAC0E0E9C0E0AB63AA64A965756C
:10263100F010E53FA4F58285F083120C54FD754935
:1026410000754A00754B43D0E0F9D0E0FAD0E0FBC9
:10265100122521053F80940540808512250AE478E2
:0226610080F601
:012663002254
:022422008F3EEB
:10242400E4F544F545F541F54A754B00754C44FB1C
:102434007A00798C7D16122A9C122A8BE543643427
:102444007004E54264127003434101E4F540E54041
:10245400C3781D9640030224F5E4F53FAB63AA64F8
:10246400A96575F010E53FA4F58285F083120C543C
:10247400607AE53E6054E53F75F010A429F9EA3529
:10248400F0FA90000D120F107889E68540F0A42927
:10249400F9EA35F0FAEBC0E0EAC0E0E9C0E0AB638A
:1024A400AA64A96575F010E53FA4F58285F083124E
:1024B4000C54FD754A00754B00754C44D0E0F9D0BE
:1024C400E0FAD0E0FB122A9C801DAB63AA64A965E4
:1024D40075F010E53FA4F58285F083120C54254570
:1024E400F545E43544F544053F02246005400224E3
:1024F40052122A8BE54364347004E542641270037B
:05250400434102AF415C
:0125090022AF
:10087100020C26E86480F8E933E83360110460F083
:10088100ED33EC337009E8FCE9FDEAFEEBFF2204ED
:1008910060DED3EB9FEA9EE99DE8C2E78CF0C2F7E8
:1008A10095F0400CE8CCF8E9CDF9EACEFAEBCFFBB4
:1008B100120BF185D0F05804700320D5B3E8047011
:1008C100075002B2D5020C3092D5EC0460F7E4CCAB
:1008D100C0E0C398F8603B94186008400DD0E0FB7D
:1008E100020C08E4FBFAC9FC8028E830E406E4C9FC
:1008F100FBE4CAFCE830E305E4C9CACBFCE85407D1
:100901006010F8C3E913F9EA13FAEB13FBEC13FCDB
:10091100D8F130F52FC3E49CFCEF9BFFEE9AFEED7E
:1009210099FDD0E0FBEF4E4D4C701222DB03020C1F
:100931002DEC2CFCEF33FFEE33FEED33FDED30E714
:10094100EB020C08EF2BFFEE3AFEED39FDD0E0FB98
:1009510050130BBB0003020C30ED13FDEE13FEEF41
:0809610013FFEC13FC020C086B
:10096900EC4D6011E8497017ED33EC3304600DE488
:10097900FCFFFEFD22E933E8330470F8020C26126D
:100989000BF158046009E4CC24815006285009026F
:100999000C30284003020C2DC0E0EB4A7044B980AA
:1009A90006D0E0FB020C1CEF4E701CBD8008EBFF6B
:1009B900EAFEE9FD80EBE98DF0A4FEE5F0020A52BA
:1009C900E9CDF9EAFEEBFFEF89F0A4FCE5F0CE8969
:1009D900F0A42EFFE435F0CD89F0A42DFEE435F026
:1009E9008067EF4E7005BD80D780C3EF8BF0A4AC54
:1009F900F0EE8BF0A42CFCE435F0F8EF8AF0A42C8F
:100A0900E5F038FCE433CB8DF0A42CFCE5F03BF8A1
:100A1900EE8AF0A42CFCE5F038F8E433CF89F0A491
:100A29002CFCE5F038CF3400CE89F0A42FFFE5F097
:100A39003EFEE433C98DF0A42EFEE5F039CD8AF0EF
:100A4900A42FFFE5F03EFEE43DFD33D0E0FB500767
:100A59000BBB000F020C30EC2CFCEF33FFEE33FE26
:060A6900ED33FD020C0854
:100A6F00020C30EC5D046005E859047003020C269B
:100A7F00120BF1580460F6EC4860F2EC7004FDFEC6
:100A8F00FF22C860DB2481C85009C398600250065A
:100A9F00020C2D9850CAF582E9294B4A7005AB829A
:100AAF00020C1C75F0007C1A7880C3EF9BEE9AED58
:100ABF0099400DC3EF9BFFEE9AFEED99FDE842F0D2
:100ACF00DC23ACF0D0E0FFD0E0FED0E0FDAB822025
:100ADF00E7101BEB60BAEC2CFCEF33FFEE33FEEDAF
:100AEF0033FD020C08E803F830E705C0F075F0009D
:100AFF00EF2FFFEE33FEED33FD40B830E7C280AA93
:100B0F0074F8CC6480CCC86480C8F582046043C399
:100B1F00EB9FF5F0EA9E42F0E99D42F0E89C45F02C
:100B2F0060305018E5825FFFE582F42B5582FB5051
:100B3F00210ABA001D09B90019088016E5825BFB6E
:100B4F00E582F42F5582FF50090EBE00050DBD0042
:100B5F00010CC3EB9FF5F0EA9E42F0E99D42F0E8ED
:0D0B6F009C45F06007CC4820E701B3EC2264
:100B7C0075F020800E75F010800575F0087D007EF4
:100B8C00007F003392D530D503120E83EC33401026
:100B9C00EF33FFEE33FEED33FDEC33FCD5F0ED22FD
:0E0BAC00E5F0247EA2D513CC92E7CDCEFF2239
:100BBA00EDD2E7CD33EC3392D524814006E4FFFE33
:100BCA00FDFC22FCE4CFCECDCC24E0501174FF8092
:100BDA00EDC3CC13CCCD13CDCE13CECF13CF04702F
:070BEA00F030D5DE020E839E
:100BF100E9D2E7C933E833F892D5EDD2E7CD33EC4A
:070C010033FC5002B2D522C2
:100C0800EC30E7100FBF000C0EBE00080DBD00044D
:100C18000BEB6014A2D5EB13FCED92E7FD2274FFF9
:100C2800FCFDFEFF22E480F8A2D574FF13FC7D8052
:030C3800E480EF66
:03000000022823B0
:0C282300787FE4F6D8FD7581BD02286ABC
:100C3B00BB010689828A83E0225002E722BBFE02B7
:090C4B00E32289828A83E49322EA
:100C5400BB010CE58229F582E5833AF583E0225055
:100C640006E92582F8E622BBFE06E92582F8E2229F
:0D0C7400E58229F582E5833AF583E49322B9
:100C8100BB010689828A83F0225002F722BBFE0152
:020C9100F3224C
:100C9300F8BB010DE58229F582E5833AF583E8F097
:100CA300225006E92582C8F622BBFE05E92582C843
:020CB300F2222B
:100CB500EF8DF0A4A8F0CF8CF0A428CE8DF0A42E53
:020CC500FE220D
:100CC700BC000BBE0029EF8DF084FFADF022E4CC11
:100CD700F875F008EF2FFFEE33FEEC33FCEE9DECDA
:100CE700984005FCEE9DFE0FD5F0E9E4CEFD22ED20
:100CF700F8F5F0EE8420D21CFEADF075F008EF2F6A
:100D0700FFED33FD4007985006D5F0F222C398FD5A
:050D17000FD5F0EA22F7
:100D1C00C2D5EC30E709B2D5E4C39DFDE49CFCEEF2
:100D2C0030E715B2D5E4C39FFFE49EFE120CC7C397
:100D3C00E49DFDE49CFC8003120CC730D507C3E492
:060D4C009FFFE49EFE2261
:100D5200BB010A89828A83E0F5F0A3E0225006876C
:100D6200F009E71922BBFE07E3F5F009E31922892E
:0B0D7200828A83E493F5F07401932261
:100D7D00BB010789828A83020F92500B09C5F027A8
:100D8D00F7C5F01937F722BBFE0D09F8E325F0F38F
:100D9D00C5F019E338F322F889828A83740193250B
:080DAD00F0C5F0F8E4933822D0
:100DB50075F008758200EF2FFFEE33FECD33CDCCF5
:100DC50033CCC58233C5829BED9AEC99E582984078
:100DD5000CF582EE9BFEED9AFDEC99FC0FD5F0D655
:100DE500E4CEFBE4CDFAE4CCF9A88222B800C1B97F
:100DF5000059BA002DEC8BF084CFCECDFCE5F0CBBD
:100E0500F97818EF2FFFEE33FEED33FDEC33FCEBF5
:100E150033FB10D703994004EB99FB0FD8E5E4F9B0
:100E2500FA227818EF2FFFEE33FEED33FDEC33FC9D
:100E3500C933C910D7059BE99A4007EC9BFCE99A91
:100E4500F90FD8E0E4C9FAE4CCFB2275F010EF2FD6
:100E5500FFEE33FEED33FDCC33CCC833C810D707D6
:100E65009BEC9AE899400AED9BFDEC9AFCE899F811
:0E0E75000FD5F0DAE4CDFBE4CCFAE4C8F922A4
:0E0E8300C3E49FFFE49EFEE49DFDE49CFC2280
:100E9100EB9FF5F0EA9E42F0E99D42F0E89C45F0B7
:010EA100222E
:0C0EA200E6FC08E6FD08E6FE08E6FF227C
:0C0EAE00ECF608EDF608EEF608EFF62270
:0C0EBA00ECF0A3EDF0A3EEF0A3EFF022AB
:100EC600D083D082E493F608740193F608740293F3
:090ED600F608740393F67404732A
:100EDF00A8828583F0D083D082120EF6120EF612FE
:100EEF000EF6120EF6E473E493A3C583C5F0C58323
:100EFF00C8C582C8F0A3C583C5F0C583C8C582C85D
:010F0F0022BF
:100F1000BB010DE58229F582E5833AF583020FB125
:100F20005007E92582F8020FA8BBFE07E92582F8E1
:100F3000020FBAE58229F582E5833AF583020FC3F1
:100F4000D083D082F8E4937012740193700DA3A340
:100F500093F8740193F5828883E473740293686054
:060F6000EFA3A3A380DF54
:102BFD008B3E8A3F8940E4F546F547E5451545AEE0
:102C0D0044700215444E6033AB41AA42A943120CE5
:102C1D003BFFAB3EAA3FA9400547E547AC467002D6
:102C2D00054614F5828C83EF120C93EF60CD740181
:102C3D002543F543E43542F54280C0AB3EAA3FA99A
:022C4D00402223
:100F6600EF4E6012EF60010EEDBB010B89828A83A2
:100F7600F0A3DFFCDEFA2289F05007F709DFFCA9AF
:0C0F8600F022BBFEFCF309DFFCA9F02206
:10282F00022EAAE493A3F8E493A34003F68001F2E7
:10283F0008DFF48029E493A3F85407240CC8C333AA
:10284F00C4540F4420C8834004F456800146F6DF79
:10285F00E4800B0102040810204080902E7FE47E5C
:10286F00019360BCA3FF543F30E509541FFEE4936E
:10287F00A360010ECF54C025E060A840B8E493A335
:10288F00FAE493A3F8E493A3C8C582C8CAC583CA60
:10289F00F0A3C8C582C8CAC583CADFE9DEE780BE18
:012E90000041
:100F9200C5F0F8A3E028F0C5F0F8E58215827002EA
:060FA2001583E038F02287
:090FA800E6FB08E6FA08E6F9226E
:090FB100E0FBA3E0FAA3E0F92241
:090FBA00E2FB08E2FA08E2F92268
:0C0FC300E493FB740193FA740293F9228A
:00000001FF
